:1000000009298030A100FE30A7200130A7207530DB
:10001000A7003030BE28A101A117AF00AF08031D13
:100020001328030114280130AF020310A20CA20C04
:10003000A20CC0302205403EAF07FE30A7202F089B
:10004000A728A101A117AF00FE30A7202F08A728DD
:10005000A401AA00AB01A01124080319A0150530C2
:10006000A3002730A900103041200330A900E83058
:100070004120A90164304120A9010A3041202A0809
:100080004828A8002B08A7002A08A600D220260886
:10009000A600A3030319A011240803195228230260
:1000A000031859282608031DA011A0195928303E0D
:1000B000A7280800AD0006118611831606118611C7
:1000C0000F30860583122D08A01884283E30A70023
:1000D0008030BE203330AC0098201330A700883029
:1000E000BE2098206430BD2098206430BD2022308E
:1000F000AC009820283083200C30832006308320E9
:10010000A0142D0884282014AC00201C92288611ED
:10011000033C031C972897200530A700DC30BE2045
:10012000031408002014FE3C0319A5288615201C82
:10013000201006150F3086052C08F03986040611AC
:10014000AC0E201898283230BD202D080429A11BA0
:100150005A2883178001840AFF3E031DAA28042918
:10016000A901A800FF30A807031CA907031C042944
:100170000330A700DF30BE20B228A701E83EA6006A
:10018000A709FC30031CC728A6070318C428A60724
:100190000000A70FC4282618CD28A61CD1280000CF
:1001A000D1280800AB01AA011030AC00270DAA0D20
:1001B000AB0D2808AA022908031C290FAB0203185B
:1001C000E8282808AA0729080318290FAB070310F5
:1001D000A60DA70DAC0BD628260804291030B000B8
:1001E000A701A601AD0CAC0C031CFC282808A6072F
:1001F00029080318290FA707A70CA60CAB0CAA0CFB
:10020000B00BF2282A080429831383120313000079
:100210000800A00107309F00E03083168500FF3002
:1002200086008113831285018601203084006030AE
:10023000AA20A03084005030AA2020308400303022
:10024000A920C830B020012077305A205A205A20E7
:100250002E305A2070305A2069305A2063305A208C
:1002600062305A2061305A2073305A2069305A2047
:1002700063305A202E305A206E305A206C305A206B
:100280000B30A900B830B120012044305A2043304F
:100290005A2046305A2032305A2030305A205530B9
:1002A0005A204B305A2041305A2020305A205A20B0
:1002B00056305A202D305A2032305A200730A900AB
:1002C000D030B120012041305A2064305A206A30A9
:1002D0005A2075305A2073305A2074305A202030FA
:1002E0005A204C305A2044305A2052305A20861816
:1002F0007F29851F7D2905147E2905107729012076
:1003000053305A2065305A2061305A2072305A20BA
:1003100063305A2068305A2020305A2073305A20D7
:1003200069305A2067305A206E305A2061305A2086
:100330006C305A2036140512831605128312232AB4
:10034000C3013C03A500C90149082502031CB929C2
:10035000DC21B61CB7294308A6004908A200A60163
:10036000A20A0314A60DA20BB2292608C304C90FC2
:10037000A429B2014308B100B20CB10CB20CB10C0B
:10038000B20CB10CB20CB10C0F30B2053208AD009A
:100390003108AC00A9010A30A800EE20B1002B08FA
:1003A000B200B4014308B3000F30B3050030B40508
:1003B00031083307C3000800BA01B9010618F12952
:1003C0000130B020B90A0319BA0A0B303A02031CF3
:1003D000F029031DEF29B9303902031CF029A02CA4
:1003E000DE299B30B0200618B614061CB610361C49
:1003F0000D2AAD014408AC00A9011430A800EE207C
:10040000B1002B08B2003208A7003108A600A901EC
:100410003A30A800D220BD00162A03013619013E49
:10042000B618013A03193611031D3615C40A85148E
:100430000130A900F430B1208510A901F030A800E6
:100440002808B1200800BB01C4013612361AB12AAF
:10045000BA01B901061C3D2AB90A0319BA0A0130CA
:10046000B020AF303A02031C3C2A031D3B2AC9309E
:100470003902031C3C2AA02C2A2ABA01B901061809
:100480006F2AB90A0319BA0A0A30B0203618632A4B
:1004900039080B3A3A04031D4E2A622A3908193AE0
:1004A0003A04031D552A8514622A39084B3A3A0446
:1004B000031D5C2A8510622A3908FA3A3A04031DA2
:1004C000622AA02C6E2A11303A02031C6E2A031DE8
:1004D0006D2A95303902031C6E2AA02C3F2A413028
:1004E0003B02031C742AA02CBB0A3A08031D7C2A79
:1004F00065303902031C7D2A3616361CB02AAD0140
:100500003B08AC00A9011430A800EE20B1002B0874
:10051000B2003208A7003108A600A9014130A800A6
:10052000D220BD008030A1008030212046305A20EA
:100530006F305A2075305A206E305A2064305A205D
:1005400020305A2073305A2069305A2067305A20A0
:100550006E305A2061305A206C305A2020305A2098
:10056000262A361CCD2A012049305A206E305A20C6
:1005700069305A2074305A2069305A2061305A202C
:100580006C305A2069305A207A305A2065305A200F
:100590002E305A205A205A20322B0F30BD00013005
:1005A000A2003D080B20A101B61DE52A3B30410207
:1005B0000318DC2AC10AE42AC101173045020318D6
:1005C000E32AC50AE42AC501E92A4208C10046080F
:1005D000C500051BF92A4508031DF12A0C30C70088
:1005E000F82A0D304502031CF82A0C304502C700DA
:1005F000FD2A4508C70020305A200A304702031858
:10060000032B20305A208030A100470828203A30A0
:100610005A200230A40041082920051B1B2B0C3056
:1006200045020318162B61305A20182B70305A20BF
:100630001230BD001D2B1330BD00410803190130DD
:10064000031D0301B5001E30410203190130031DD3
:1006500003013504B5000130861803013504031980
:10066000322B782C361E762CDC210130C9000F305D
:10067000490203183E2BDC21C90F372B3611B61166
:10068000DC21DC21DC21B61C472B0514482B05108E
:100690001230C900143049020318512BDC21C90F54
:1006A0004A2BDC210730BC00A0214308C200DC211A
:1006B000361D5B2BB6150630BC00A0214308C600D2
:1006C000DC21361D642BB6150630BC00A021430882
:1006D000BE000330BC00A0214308C8000530BC00A8
:1006E000A0214308C0000830BC00A0214308BF007F
:1006F000DC21361D7C2BB615361C822BB619812BBE
:1007000036100120B619752C80302120A10101304E
:100710004802031D922B4D305A206F305A206E3004
:100720005A20D32B02304802031D9D2B54305A20EF
:1007300075305A2065305A20D32B03304802031DF0
:10074000A82B57305A2065305A2064305A20D32BBA
:1007500004304802031DB32B54305A2068305A200D
:1007600075305A20D32B05304802031DBE2B46306E
:100770005A2072305A2069305A20D32B0630480252
:10078000031DC92B53305A2061305A2074305A202F
:10079000D32B07304802031DD32B53305A2075301A
:1007A0005A206E305A208030A100843021203E082B
:1007B000282020305A2001304002031DE62B4A3009
:1007C0005A2061305A206E305A205E2C023040028E
:1007D000031DF12B46305A2065305A2062305A20D2
:1007E0005E2C03304002031DFC2B4D305A2061303B
:1007F0005A2072305A205E2C04304002031D072C10
:1008000041305A2070305A2072305A205E2C053008
:100810004002031D122C4D305A2061305A2079308D
:100820005A205E2C06304002031D1D2C4A305A20EF
:1008300075305A206E305A205E2C07304002031D5E
:10084000282C4A305A2075305A206C305A205E2CA1
:1008500008304002031D332C41305A2075305A2095
:1008600067305A205E2C09304002031D3E2C533065
:100870005A2065305A2070305A205E2C0A304002CF
:10088000031D492C4F305A2063305A2074305A20AF
:100890005E2C0B304002031D542C4E305A206F301A
:1008A0005A2076305A205E2C0C304002031D5E2CFC
:1008B00044305A2065305A2063305A20051B6B2C77
:1008C00020305A208030A1000230A4003F082920A7
:1008D00020305A20752C20305A2027305A20803062
:1008E000A1000230A4003F082920772CA02C232A45
:1008F000851F7F2C0512831605128312812C831607
:10090000051683129B30B020410803190130031DE6
:100910000301B50001308618030135040319912C39
:100920000515851585140130A900F430B120051195
:10093000851185100130A9004A30B120C40A352B39
:1009400001204E305A206F305A2020305A20733008
:100950005A2069305A2067305A206E305A20613050
:100960005A206C305A20203084006030AA20A030F9
:1009700084005030AA20203084003030A92006188E
:10098000B616061CB61203010618013EB61A013C43
:10099000031DD02CB70A0319B80A0130B020C32CAC
:1009A0000301B61A0130013A0319B612031DB61637
:1009B00003010618013EB61A013C031DE52CB70AD7
:1009C0000319B80A0130B020D82C03303802DE30C9
:0C09D000031937020318B32C3614232A35
:02400E00503F21
:00000001FF
